:020000040000FA
:0A0000000000000025EF00F03CD0E6
:0800180089D0096A086EFF0E91
:100020000826092200D0D8A01200030E076EE60EA3
:1000300002D8F5D7076AFE0F066EE86A075AD8A0FD
:1000400012000000060600D0F8D74F0EAF6E240E47
:10005000AC6E900EAB6E00010FEE7FF0ED6AE950D2
:10006000EA10FCE1EF6A0F0EC16E070EB46EC69A7D
:10007000C30E926EE00E936EC00E946E92809282CA
:100080006ED0F2A403D0F294817A11009EAA19D006
:10009000060EAB1412E1E2CF31F0E1CF30F0322A9C
:1000A00010EE54F03250E126000EE222AECFE7FF10
:1000B00031C0E2FF30C0E1FF1100AE50AE50AB984E
:1000C000AB8811003250335C14E0332AEACF07F0DA
:1000D000E9CF06F000EE54F03350E926000EEA2294
:1000E000EF50066E07C0EAFF06C0E9FFD880120095
:1000F00004D0E868066ED8A012001200326A336A93
:100100009D8A9F8AF28EF28C12009D9A00EE54F026
:10011000010EF46EF36AF306000EF45AEE6AF45020
:10012000F310F9E1326A336A9D8A1200F29EE0CF41
:1001300054F4D8CF55F4E8CF56F4F28E0001A192D2
:10014000B36AB26AF29E54C4E0FF55C4D8FF56C4E5
:10015000E8FFF28E10009EA8FED7AD6E1200939AB3
:100160008A8A0A0E5ADF939A8A9A9296899693946B
:100170008A9492948994949A8B9A94988B98949652
:100180008B9694948B9494928B9294908B90929A59
:10019000899A929889981B6A196A00EE34F0200EA9
:1001A000EE68E82EFDD71A6AA9DFAFDFCD6AF294B8
:1001B000F28A870ED56EB16AA192A082B36AB26A42
:1001C000D08EA292B10EB16E3BEC06F038EC0AF084
:1001D000292AE86A29B2010F2AB0010806E12A702B
:1001E000252A000E2622272228226CDF0A6EED0E19
:1001F0000A5C06E3FE0E0A5C01E20C6AECEF03F017
:100200000AAE38D00C6A8C0E0A5C05E10AC00CF00C
:100210000D680E682DD09C0E0A5C05E10AC00CF03A
:100220000F68106825D0AC0E0A5C05E10AC00CF01E
:10023000116812681DD0BC0E0A5C05E10AC00CF002
:100240001368146815D0CC0E0A5C04E10AC00CF0E7
:1002500015680ED0DC0E0A5C04E10AC00CF01668CA
:1002600007D0EC0E0A5C04E10AC00CF017681868AD
:10027000EBEF03F00C5204E1ECEF03F0EBEF03F0D3
:100280008C0E0C5CD8A468D00D2803E10AC00DF0D8
:100290005FD00AC00EF0780E0D5C08E18B9A1990C1
:1002A0001B9037683668356834684FD0790E0D5C1E
:1002B00008E18B9819921B923B683A683968386854
:1002C00044D07A0E0D5C08E18B9619941B943F681C
:1002D0003E683D683C6839D07B0E0D5C08E18B942C
:1002E00019961B9643684268416840682ED07C0E80
:1002F0000D5C08E18B9219981B9847684668456821
:10030000446823D07D0E0D5C08E18B90199A1B9AEE
:100310004B684A684968486818D07E0E0D5C08E151
:10032000899A199C1B9C4F684E684D684C680DD08B
:100330007F0E0D5C08E18998199E1B9E53685268D8
:100340005168506802D0ECEF03F00D68EBEF03F05A
:10035000ECEF03F0EBEF03F09C0E0C5CD8A4FDD1A6
:100360000F2803E10AC00FF0F6D10AC010F01052B6
:10037000D8A45BD0780E0F5C08E18B9A19901B9083
:1003800037683668356834684ED0790E0F5C08E1FE
:100390008B9819921B923B683A683968386843D049
:1003A0007A0E0F5C08E18B9619941B943F683E68A7
:1003B0003D683C6838D07B0E0F5C08E18B94199641
:1003C0001B9643684268416840682DD07C0E0F5CE4
:1003D00008E18B9219981B984768466845684468FD
:1003E00022D07D0E0F5C08E18B90199A1B9A4B6806
:1003F0004A684968486817D07E0E0F5C08E1899A00
:10040000199C1B9C4F684E684D684C680CD07F0E41
:100410000F5C08E18998199E1B9E536852685168C9
:10042000506801D0D9D1D7D196D11AA092D1780EE7
:100430000F5C2FE110C01DF08B8A7F0E1D5C22E245
:100440001B8002EE54F0D8901D34E926000EEA22FB
:10045000EECF04F0EFCF05F004502524006E0550D8
:100460002620016E000E2720026E000E2820036E4B
:1004700003C037F002C036F001C035F000C034F0E0
:10048000198006D01B901990376836683568346833
:1004900060D1790E0F5C2FE110C01EF08B887F0EAB
:1004A0001E5C22E21B8202EE54F0D8901E34E92634
:1004B000000EEA22EECF04F0EFCF05F00450252421
:1004C000006E05502620016E000E2720026E000EE1
:1004D0002820036E03C03BF002C03AF001C039F09F
:1004E00000C038F0198206D01B9219923B683A6816
:1004F000396838682ED17A0E0F5C2FE110C01FF0DA
:100500008B867F0E1F5C22E21B8402EE54F0D89093
:100510001F34E926000EEA22EECF04F0EFCF05F0FB
:1005200004502524006E05502620016E000E272061
:10053000026E000E2820036E03C03FF002C03EF0A2
:1005400001C03DF000C03CF0198406D01B94199402
:100550003F683E683D683C68FCD07B0E0F5C2FE135
:1005600010C020F08B847F0E205C22E21B8602EEFE
:1005700054F0D8902034E926000EEA22EECF04F0A1
:10058000EFCF05F004502524006E05502620016EA3
:10059000000E2720026E000E2820036E03C043F0D9
:1005A00002C042F001C041F000C040F0198606D000
:1005B0001B9619964368426841684068CAD07C0E11
:1005C0000F5C2FE110C021F08B827F0E215C22E2B4
:1005D0001B8802EE54F0D8902134E926000EEA225E
:1005E000EECF04F0EFCF05F004502524006E055047
:1005F0002620016E000E2720026E000E2820036EBA
:1006000003C047F002C046F001C045F000C044F00E
:10061000198806D01B981998476846684568446849
:1006200098D07D0E0F5C2FE110C022F08B807F0EE2
:10063000225C22E21B8A02EE54F0D8902234E92692
:10064000000EEA22EECF04F0EFCF05F0045025248F
:10065000006E05502620016E000E2720026E000E4F
:100660002820036E03C04BF002C04AF001C049F0DD
:1006700000C048F0198A06D01B9A199A4B684A683C
:100680004968486866D07E0E0F5C2FE110C023F0E9
:10069000898A7F0E235C22E21B8C02EE54F0D890F4
:1006A0002334E926000EEA22EECF04F0EFCF05F066
:1006B00004502524006E05502620016E000E2720D0
:1006C000026E000E2820036E03C04FF002C04EF0F1
:1006D00001C04DF000C04CF0198C06D01B9C199C39
:1006E0004F684E684D684C6834D07F0E0F5C2FE128
:1006F00010C024F089887F0E245C22E21B8E02EE5B
:1007000054F0D8902434E926000EEA22EECF04F00B
:10071000EFCF05F004502524006E05502620016E11
:10072000000E2720026E000E2820036E03C053F037
:1007300002C052F001C051F000C050F0198E06D036
:100740001B9E199E536852685168506802D00F680A
:1007500043D00F6840D040D03ED0AC0E0C5C0BE1D3
:10076000112803E10AC011F004D00AC012F0FBD92D
:1007700032D032D030D0BC0E0C5C0BE1132803E138
:100780000AC013F004D00AC014F0EAEC05F024D03B
:1007900022D0CC0E0C5C08E1152804E10AC015F04B
:1007A000E4EC05F019D017D0DC0E0C5C08E116283B
:1007B00004E10AC016F0E8EC05F00ED00CD0EC0E07
:1007C0000C5C09E1172803E10AC017F003D00AC046
:1007D00018F0FCD901D08DD9080E2F5CD8B080D18B
:1007E0002B50255C2C5026582D5027582E50285819
:1007F000D8A068D12E8E2F522AE11BB006D08B9A3A
:10080000376836683568346821D0827A949A02EE67
:1008100054F0D8901D34E926000EEA22EECF04F001
:10082000EFCF05F004502524006E05502620016E00
:10083000000E2720026E000E2820036E03C037F042
:1008400002C036F001C035F000C034F03AD1010EDC
:100850002F5C2AE11BB206D08B983B683A68396856
:10086000386821D08278949802EE54F0D8901E34E3
:10087000E926000EEA22EECF04F0EFCF05F0045097
:100880002524006E05502620016E000E2720026EE2
:10089000000E2820036E03C03BF002C03AF001C0F6
:1008A00039F000C038F00DD1020E2F5C2AE11BB4E4
:1008B00006D08B963F683E683D683C6821D08276C2
:1008C000949602EE54F0D8901F34E926000EEA22E6
:1008D000EECF04F0EFCF05F004502524006E055054
:1008E0002620016E000E2720026E000E2820036EC7
:1008F00003C03FF002C03EF001C03DF000C03CF03C
:10090000E0D0030E2F5C2AE11BB606D08B9443681F
:1009100042684168406821D08274949402EE54F099
:10092000D8902034E926000EEA22EECF04F0EFCF73
:1009300005F004502524006E05502620016E000E9F
:100940002720026E000E2820036E03C043F002C071
:1009500042F001C041F000C040F0B3D0040E2F5C63
:100960002AE11BB806D08B92476846684568446800
:1009700021D08272949202EE54F0D8902134E9266C
:10098000000EEA22EECF04F0EFCF05F0045025244C
:10099000006E05502620016E000E2720026E000E0C
:1009A0002820036E03C047F002C046F001C045F0A6
:1009B00000C044F086D0050E2F5C2AE11BBA06D099
:1009C0008B904B684A684968486821D0827094903F
:1009D00002EE54F0D8902234E926000EEA22EECF3F
:1009E00004F0EFCF05F004502524006E05502620BA
:1009F000016E000E2720026E000E2820036E03C039
:100A00004BF002C04AF001C049F000C048F059D094
:100A1000060E2F5C2AE11BBC06D0899A4F684E68EF
:100A20004D684C6821D0807A929A02EE54F0D890AA
:100A30002334E926000EEA22EECF04F0EFCF05F0D2
:100A400004502524006E05502620016E000E27203C
:100A5000026E000E2820036E03C04FF002C04EF05D
:100A600001C04DF000C04CF02CD0070E2F5C29E1E6
:100A70001BBE06D08998536852685168506821D0CF
:100A80008078929802EE54F0D8902434E926000E33
:100A9000EA22EECF04F0EFCF05F004502524006EDB
:100AA00005502620016E000E2720026E000E282021
:100AB000036E03C053F002C052F001C051F000C0F9
:100AC00050F017D828AE0BD0286A276A266A256A04
:100AD0001B6A00EE34F0200EEE68E82EFDD706D03B
:100AE00028AE04D0286A276A266A256A8170E8EF52
:100AF00000F02F682E8E0B6A080E0B5C33E2D89044
:100B00000B34E96EEA6AEA36E936EA36340EE9264B
:100B1000000EEA22EFCF00F0ECCF01F0ECCF02F0B4
:100B2000ECCF03F02B50005C2C5001582D50025894
:100B30002E50035815E2D8900B34E96EEA6AEA3673
:100B4000E936EA36340EE926000EEA22EFCF2BF022
:100B5000ECCF2CF0ECCF2DF0ECCF2EF00BC02FF023
:100B60000B2ACAE31200780E115C03E112C01DF0DB
:100B700029D0790E115C03E112C01EF023D07A0E49
:100B8000115C03E112C01FF01DD07B0E115C03E16C
:100B900012C020F017D07C0E115C03E112C021F0CE
:100BA00011D07D0E115C03E112C022F00BD07E0E3D
:100BB000115C03E112C023F005D07F0E115C02E14D
:100BC00012C024F011681200156812001768120094
:100BD000166812001E0E135C11E112C01DF012C047
:100BE0001EF012C01FF012C020F012C021F012C07F
:100BF00022F012C023F012C024F026D0320E135C73
:100C000004E189861A8089841FD0330E135C04E1C5
:100C100089861A80898418D0420E135C09E1145227
:100C200003E11A9013D803D0898689841A800CD0E6
:100C30007B0E135C09E11B6A8B9A8B988B968B94C5
:100C40008B928B90899A899813681200899689945F
:100C50001B6A1D6A1E6A1F6A206A216A226A236A49
:100C6000246A8B9A8B988B968B948B928B90899A13
:100C700089981A6A12000201556954695C0E576F0F
:100C80007A0E566F590E596F850E586F580E5B6F5E
:100C9000140E5A6F560E5D6FA90E5C6F550E5F6F86
:100CA000430E5E6F530E616FE30E606F520E636F03
:100CB000890E626F510E656F350E646F4F0E676F50
:100CC000E60E666F4E0E696F9C0E686F4D0E6B6F71
:100CD000580E6A6F4C0E6D6F190E6C6F4A0E6F6F67
:100CE000DF0E6E6F490E716FAA0E706F480E736F34
:100CF0007A0E726F470E756F4F0E746F460E776FD8
:100D0000290E766F450E796F080E786F430E7B6F54
:100D1000EB0E7A6F420E7D6FD30E7C6F410E7F6FAC
:100D2000BF0E7E6F400E816FB00E806F3F0E836FDF
:100D3000A50E826F3E0E856F9E0E846F3D0E876FEF
:100D40009C0E866F3C0E896F9E0E886F3B0E8B6FDC
:100D5000A40E8A6F3A0E8D6FAE0E8C6F390E8F6FA8
:100D6000BC0E8E6F380E916FCE0E906F370E936F54
:100D7000E30E926F360E956FFD0E946F360E976FE1
:100D80001A0E966F350E996F3B0E986F340E9B6F4F
:100D90005F0E9A6F330E9D6F870E9C6F320E9F6FA2
:100DA000B20E9E6F310EA16FE10EA06F310EA36FD8
:100DB000140EA26F300EA56F490EA46F2F0EA76FF1
:100DC000820EA66F2E0EA96FBE0EA86F2D0EAB6FF2
:100DD000FD0EAA6F2D0EAD6F3F0EAC6F2C0EAF6FD8
:100DE000850EAE6F2B0EB16FCD0EB06F2B0EB36FA5
:100DF000180EB26F2A0EB56F670EB46F290EB76F5B
:100E0000B80EB66F290EB96F0C0EB86F280EBB6FF7
:100E1000620EBA6F270EBD6FBC0EBC6F270EBF6F80
:100E2000180EBE6F260EC16F760EC06F250EC36FF3
:100E3000D80EC26F250EC56F3C0EC46F240EC76F4F
:100E4000A20EC66F240EC96F0B0EC86F230ECB6F98
:100E5000760ECA6F220ECD6FE40ECC6F220ECF6FCE
:100E6000540ECE6F210ED16FC60ED06F210ED36FF0
:100E70003B0ED26F200ED56FB20ED46F200ED76FFF
:100E80002B0ED66F1F0ED96FA60ED86F1F0EDB6FFD
:100E9000240EDA6F1E0EDD6FA30EDC6F1E0EDF6FE9
:100EA000250EDE6F1D0EE16FA90EE06F1D0EE36FC4
:100EB0002E0EE26F1C0EE56FB60EE46F1C0EE76F90
:100EC0003F0EE66F1B0EE96FCB0EE86F1B0EEB6F4C
:100ED000580EEA6F1A0EED6FE80EEC6F1A0EEF6FF8
:100EE000790EEE6F1A0EF16F0B0EF06F190EF36F95
:100EF000A00EF26F190EF56F360EF46F180EF76F25
:100F0000CE0EF66F180EF96F680EF86F180EFB6FA5
:100F1000030EFA6F170EFD6FA00EFC6F170EFF6F1A
:100F20003F0EFE6F160E0301016FDF0E006F160EEF
:100F3000036F800E026F160E056F240E046F150EE0
:100F4000076FC80E066F150E096F6E0E086F150E2F
:100F50000B6F160E0A6F140E0D6FBF0E0C6F140E72
:100F60000F6F690E0E6F140E116F150E106F130EAA
:100F7000136FC20E126F130E156F710E146F130ED6
:100F8000176F210E166F120E196FD20E186F120EF8
:100F90001B6F840E1A6F120E1D6F380E1C6F110E10
:100FA0001F6FED0E1E6F110E216FA30E206F110E1D
:100FB000236F5A0E226F110E256F120E246F100E22
:100FC000276FCC0E266F100E296F870E286F100E1C
:100FD0002B6F420E2A6F0F0E2D6F2C692F6FBD0ED7
:100FE0002E6F0F0E316F7C0E306F0F0E336F3D0E74
:100FF000326F0E0E356FFE0E346F0E0E376FC00E51
:10100000366F0E0E396F830E386F0E0E3B6F470E24
:101010003A6F0E0E3D6F0C0E3C6F0D0E3F6FD20EF1
:101020003E6F0D0E416F990E406F0D0E436F610EB6
:10103000426F0D0E456F2A0E446F0C0E476FF40E73
:10104000466F0C0E496FBE0E486F0C0E4B6F8A0E2A
:101050004A6F0C0E4D6F560E4C6F0C0E4F6F230ED9
:101060004E6F0B0E516FF10E506F0B0E536FC00E83
:10107000526F55695469A20E576FC30E566F9A0E80
:10108000596F460E586F960E5B6F320E5A6F920E66
:101090005D6F3A0E5C6F8E0E5F6F5D0E5E6F8A0E37
:1010A000616F9A0E606F860E636FF00E626F830E33
:1010B000656F5F0E646F7F0E676FE70E666F7C0E65
:1010C000696F850E686F790E6B6F3B0E6A6F760ED7
:1010D0006D6F070E6C6F720E6F6FE80E6E6F6F0E96
:1010E000716FDF0E706F6C0E736FEA0E726F6A0EA7
:1010F000756F0A0E746F670E776F3C0E766F640E15
:10110000796F820E786F610E7B6FDA0E7A6F5F0EE9
:101110007D6F440E7C6F5C0E7F6FBF0E7E6F5A0E2C
:10112000816F4C0E806F570E836FE90E826F550EE4
:10113000856F960E846F530E876F866F510E896F81
:10114000200E886F4E0E8B6FFB0E8A6F4C0E8D6FCC
:10115000E50E8C6F4A0E8F6FDC0E8E6F480E916F0E
:10116000E20E906F460E936FF50E926F450E956FDF
:10117000150E946F430E976F420E966F410E996F46
:101180007B0E986F3F0E9B6FC00E9A6F3E0E9D6F49
:10119000100E9C6F3C0E9F6F6D0E9E6F3A0EA16FEE
:1011A000D40EA06F390EA36F460EA26F370EA56F37
:1011B000C20EA46F360EA76F490EA66F340EA96F2C
:1011C000DA0EA86F330EAB6F740EAA6F320EAD6FCE
:1011D000180EAC6F300EAF6FC50EAE6F2F0EB16F25
:1011E0007B0EB06F2E0EB36F3A0EB26F2D0EB56F31
:1011F000020EB46F2B0EB76FD10EB66F2A0EB96FF9
:10120000A90EB86F290EBB6F880EBA6F280EBD6F7E
:101210006F0EBC6F270EBF6F5E0EBE6F260EC16FC6
:10122000530EC06F250EC36F500EC26F240EC56FD4
:10123000540EC46F230EC76F5E0EC66F220EC96FA9
:101240006F0EC86F210ECB6F860ECA6F200ECD6F4A
:10125000A30ECC6F1F0ECF6FC60ECE6F1E0ED16FBA
:10126000EF0ED06F1E0ED36FD26F1D0ED56F520EC4
:10127000D46F1C0ED76F8C0ED66F1B0ED96FCB0E92
:10128000D86F1B0EDB6F0F0EDA6F1A0EDD6F580E64
:10129000DC6F190EDF6FA50EDE6F180EE16FF80E12
:1012A000E06F180EE36F4F0EE26F170EE56FAB0E97
:1012B000E46F170EE76F0A0EE66F160EE96F6F0EFA
:1012C000E86F150EEB6FD70EEA6F150EED6F430E3C
:1012D000EC6F140EEF6FB30EEE6F140EF16F270E5E
:1012E000F06F130EF36F9F0EF26F130EF56F1A0E61
:1012F000F46F120EF76F990EF66F120EF96F1B0E48
:10130000F86F110EFB6FA10EFA6F110EFD6F290E13
:10131000FC6F100EFF6FB50EFE6F100E0401016F13
:10132000440E006F0F0E036FD60E026F0F0E056F87
:101330006B0E046F0F0E076F030E066F0E0E096F14
:101340009D0E086F0E0E0B6F3A0E0A6F0D0E0D6F8D
:10135000DA0E0C6F0D0E0F6F7C0E0E6F0D0E116FEF
:10136000210E106F0C0E136FC80E126F0C0E156F3E
:10137000720E146F0C0E176F1E0E166F0B0E196F78
:10138000CC0E186F0B0E1B6F7C0E1A6F0B0E1D6FA1
:101390002E0E1C6F0A0E1F6FE30E1E6F0A0E216FBA
:1013A000990E206F0A0E236F510E226F0A0E256FC1
:1013B0000B0E246F090E276FC80E266F090E296FBA
:1013C000850E286F090E2B6F450E2A6F090E2D6FA3
:1013D000060E2C6F080E2F6FC90E2E6F080E316F80
:1013E0008E0E306F080E336F540E326F080E356F4D
:1013F0001C0E346F070E376FE50E366F070E396F10
:10140000AF0E386F070E3B6F7B0E3A6F070E3D6FC6
:10141000490E3C6F070E3F6F170E3E6F060E416F71
:10142000E70E406F060E436FB90E426F060E456F12
:101430008B0E446F060E476F5F0E466F060E496FA8
:10144000340E486F060E4B6F0A0E4A6F050E4D6F35
:10145000E10E4C6F050E4F6FB90E4E6F050E516FBA
:10146000930E506F050E536F6D0E526F00011200F8
:10147000040E0101576F880E566F040E596FA60EA9
:10148000586F040E5B6FB60E5A6F040E5D6FC60E7A
:101490005C6F040E5F6FD60E5E6F040E616FE60E1A
:1014A000606F040E636FF60E626F050E656F070EB8
:1014B000646F050E676F170E666F050E696F280E55
:1014C000686F050E6B6F390E6A6F050E6D6F4B0EF0
:1014D0006C6F050E6F6F5D0E6E6F050E716F6E0E89
:1014E000706F050E736F800E726F050E756F930E21
:1014F000746F050E776FA50E766F050E796FB80EB7
:10150000786F050E7B6FCB0E7A6F050E7D6FDF0E49
:101510007C6F050E7F6FF20E7E6F060E816F806FFF
:10152000836F1A0E826F060E856F2E0E846F060E65
:10153000876F430E866F060E896F580E886F060EF2
:101540008B6F6D0E8A6F060E8D6F830E8C6F060E7D
:101550008F6F980E8E6F060E916FAE0E906F060E07
:10156000936FC40E926F060E956FDB0E946F060E8E
:10157000976FF20E966F070E996F090E986F070E10
:101580009B6F210E9A6F070E9D6F380E9C6F070E92
:101590009F6F500E9E6F070EA16F690EA06F070E12
:1015A000A36F810EA26F070EA56F9A0EA46F070E90
:1015B000A76FB40EA66F070EA96FCD0EA86F070E0A
:1015C000AB6FE70EAA6F080EAD6F020EAC6F080E80
:1015D000AF6F1D0EAE6F080EB16F380EB06F080EF4
:1015E000B36F530EB26F080EB56F6F0EB46F080E67
:1015F000B76F8B0EB66F080EB96FA70EB86F080ED7
:10160000BB6FC40EBA6F080EBD6FE10EBC6F080E43
:10161000BF6FBE69090EC16F1D0EC06F090EC36F8B
:101620003B0EC26F090EC56F5A0EC46F090EC76F0D
:10163000790EC66F090EC96F990EC86F090ECB6F70
:10164000B90ECA6F090ECD6FD90ECC6F090ECF6FD0
:10165000FA0ECE6F0A0ED16F1B0ED06F0A0ED36F2B
:101660003D0ED26F0A0ED56F5F0ED46F0A0ED76F84
:10167000820ED66F0A0ED96FA50ED86F0A0EDB6FD9
:10168000C80EDA6F0A0EDD6FEC0EDC6F0B0EDF6F2B
:10169000110EDE6F0B0EE16F360EE06F0B0EE36F77
:1016A0005B0EE26F0B0EE56F810EE46F0B0EE76FC2
:1016B000A70EE66F0B0EE96FCE0EE86F0B0EEB6F09
:1016C000F50EEA6F0C0EED6F1D0EEC6F0C0EEF6F4A
:1016D000460EEE6F0C0EF16F6F0EF06F0C0EF36F87
:1016E000980EF26F0C0EF56FC20EF46F0C0EF76FC2
:1016F000ED0EF66F0D0EF96F180EF86F0D0EFB6FF5
:10170000430EFA6F0D0EFD6F700EFC6F0D0EFF6F26
:101710009C0EFE6F0D0E0201016FCA0E006F0D0EC2
:10172000036FF80E026F0E0E056F260E046F0E0E7D
:10173000076F550E066F0E0E096F850E086F0E0EA1
:101740000B6FB60E0A6F0E0E0D6FE70E0C6F0F0EBD
:101750000F6F180E0E6F0F0E116F4B0E106F0F0ED6
:10176000136F7E0E126F0F0E156FB10E146F0F0EEA
:10177000176FE60E166F100E196F1B0E186F100EF6
:101780001B6F500E1A6F100E1D6F870E1C6F100E00
:101790001F6FBE0E1E6F100E216FF60E206F110E02
:1017A000236F2E0E226F110E256F680E246F110EFF
:1017B000276FA20E266F110E296FDC0E286F120EF6
:1017C0002B6F180E2A6F120E2D6F540E2C6F120EE7
:1017D0002F6F910E2E6F120E316FCF0E306F130ED2
:1017E000336F0E0E326F130E356F4D0E346F130EB6
:1017F000376F8E0E366F130E396FCF0E386F140E93
:101800003B6F110E3A6F140E3D6F540E3C6F140E69
:101810003F6F980E3E6F140E416FDC0E406F150E39
:10182000436F220E426F150E456F680E446F150E02
:10183000476FB00E466F150E496FF80E486F160EC3
:101840004B6F410E4A6F160E4D6F8C0E4C6F160E7D
:101850004F6FD70E4E6F170E516F230E506F170E2E
:0C186000536F700E526F00011200FFD792
:020000040030CA
:0300010006160ED2
:020005008580F4
:060008000FC00FE00F40E5
:00000001FF
